:0200000480007A
:100000006F00C004732F2034930F8000630AFF0336
:10001000930F90006306FF03930FB0006302FF038A
:10002000170F0000130F0F1763040F0067000F0076
:10003000732F203463540F006F00400093E19153FD
:10004000171F000023203FFC6FF09FFF732540F136
:1000500063100500970200009382020173905230F2
:10006000735000189702000093820202739052307E
:10007000B70200809382F2FF7390023B9302F0017B
:100080007390023A9702000093828201739052307B
:100090007350203073503030735040309301000063
:1000A00097020000938242F67390523013051000BD
:1000B0001315F501634C05000F00F00F93011000BC
:1000C0009308D005130500007300000093020000A0
:1000D000638E020073905210B7B2000093829210A8
:1000E0007390223073232030E39A62F4735000300F
:1000F00037250000130505807320053097020000A6
:100100009382420173901234732540F173002030C2
:100110009301200013038000B72200009382028025
:1001200073B00230F3230030B3F272006384020034
:100130001303B000B72200009382028073B0023034
:1001400097020000938202017390123473002030F2
:1001500093011000730000006F00800063103002F4
:100160000F00F00F638001009391110093E11100E3
:100170009308D00513850100730000000F00F00FF5
:10018000930110009308D0051305000073000000D0
:10019000F3222034E39662FC970300009383C3FBB1
:1001A000F3221034E39E72FA6FF05FFD731000C00B
:1001B000000000000000000000000000000000003F
:1010000000000000000000000000000000000000E0
:1010100000000000000000000000000000000000D0
:1010200000000000000000000000000000000000C0
:1010300000000000000000000000000000000000B0
:081040000000000000000000A8
:040000058000000077
:00000001FF
